:020000040000FA
:0400000085284430DB
:08000800A000030EA100831209
:100010000C1C2328DD1B23288E015C1C15285C107A
:1000200050088F005D0985051B285C1451088F005E
:100030005D088504DC170C108B180828210E83003E
:10004000A00E200E090005192B2883160117831214
:10005000B23081005D288316011383120B193728F3
:10006000AE17280A03192E17AE1948285628AE13C2
:10007000AE1945282E1F5628AE1A5628A701A601EC
:10008000A501A801AE01AE165D28F030AE055D28D1
:100090002D152E13AE122708AB002608AA0025083E
:1000A000A9002808AC00F030AE055D282E0DA80D83
:1000B000A50DA60DA70DAE1AAE0A8B100B11210EC1
:0800C0008300A00E200E0900D0
:06010A002030840080019A
:10011000840A80300402031C8728772283160C305F
:10012000850587018312850187010730990000301A
:100130009A00103083168E008312603083168F0071
:1001400083120030831691009F008312C8308316FB
:100150008100831201309000A63096001830910083
:100160008030970007309300013083168C00831293
:1001700010308B00382381018E018F010B118B1001
:100180000B108C010B178B17D9202D19DB20701841
:10019000C4284722B30BD728031085190314BA0DBE
:1001A000F0303A020319BF21F308031999261E24DF
:1001B000C428640008003F257018080029083F3C47
:1001C0000319EA282B082A0629062C02031D2D11E3
:1001D000031D08002D110130B7008B1320303707A5
:1001E00083169B001C141A088312A40010303707D2
:1001F00083169B001C141A088312A30000303707D3
:1002000083169B001C141A088312A2008B17240863
:100210002B02031DB92923082A02031DB929013025
:100220003702031D492929083F3C03193329A91B1B
:100230001F29291F1F2929081F39AF00AF17403078
:100240002906E039031D29293F1F29293F13AD172E
:10025000372960302906E039031D37293F1B37292C
:100260003F17AD173729AC1F3F13AC1B3F1780302A
:100270002906F039031D4029BF1F4029BF13AD17C0
:1002800090302906F039031D4929BF1B4929BF17A2
:10029000AD17A91FB929291BB92922082906F03948
:1002A000A91EE039031DB929220829050F390319B0
:1002B000862901303702031D62293E1862293E1447
:1002C000AD17A82202303702031D6B29BE186B2917
:1002D000BE14AD17C32203303702031D74293E1923
:1002E00074293E15AD17DE2204303702031D7D2927
:1002F000BE197D29BE15AD17F92205303702031D41
:1003000086293E1A86293E16AD171423290922058F
:100310000F390319B92901303702031D94293E1CF6
:1003200094293E10AD171E2302303702031D9D296C
:10033000BE1C9D29BE10AD17222303303702031DBA
:10034000A6293E1DA6293E11AD17262304303702EB
:10035000031DAF29BE1DAF29BE11AD172A230530DD
:100360003702031DB8293E1EB8293E12AD172E23B1
:10037000B929B70A0630370203180800ED2808002B
:100380000B13DD17B601B3019630B4000130B50090
:100390000130B70085018701AD132C22D920B30BA2
:1003A000EB29031085190314BA0DF0303A02031932
:1003B0001A2AB41F8501B41F8701B40BEB29370833
:1003C000B6080319B6000319E929FF308500870034
:1003D000B6039630B4002D1DCE292D11A91FCE29AC
:1003E000291BCE29A91E29120F3029050319CE2950
:1003F000B9012918B90AA918B90A2919B90AA919F4
:10040000B90AB918CE293919CE298B1320303707EC
:10041000BC002B08BB00572210303707BC002A084D
:10042000BB00572200303707BC002908BB00572209
:100430008B17262285018701B70AB60106303702DD
:10044000031CCE290B17DD133823080005303702B3
:1004500003190800850187011430B90033308F1F5C
:1004600085008F1B8501D9202D1D2E2A2D11290ACB
:1004700003193E2AA91F2E2A291B2E2A0F302905CF
:10048000031D2C2AB90B2E2A8501870108005C1C4C
:100490000800AD1F0800AD131030BC003E08BB00C3
:1004A00057223030BC003F08BB00572208003C08F0
:1004B0008B1383169B001C141A0883128B173B02A4
:1004C000031908008B133B0883161C159A0083122E
:1004D0003C0883169B0055309D00AA309D009C145B
:1004E00064009C18702A1C1183128B1708000A30B4
:1004F000DE007D30DF00831600309B001C141A08DC
:100500008312BD00831610309B001C141A0883123E
:10051000BE00831630309B001C141A088312BF00E3
:100520006230F100E8267208C0006330F100E8266E
:10053000720840020319F0166D30F100E8267208C7
:10054000E1006118BE016118BF010430F30008002A
:100550008B13831673309B001C141A088312C1007E
:100560008B1752100E303E05031D08008B138316A7
:100570006F309B001C141A088312C5008B178E0164
:100580008F010C1008008B13831673309B001C1412
:100590001A088312C2008B17D2100D303E05031DBE
:1005A00008008B1383166F309B001C141A088312EB
:1005B000C5008B178E018F010C1008008B1383165A
:1005C00073309B001C141A088312C3008B1752113E
:1005D0000B303E05031D08008B1383166F309B0004
:1005E0001C141A088312C5008B178E018F010C1082
:1005F00008008B13831673309B001C141A08831297
:10060000C4008B17521207303E05031D08008B13E0
:1006100083166F309B001C141A088312C5008B17B9
:100620008E018F010C1008008B13831671309B0014
:100630001C141A088312CF008B170800E61F8512BE
:10064000DD120800E71F05125D120800E81F851083
:10065000DD100800E91F05105D1008008B138316DC
:1006600072309B001C141A088312CF008B170800ED
:10067000C101C201C301C4013E1E2E2B142B080070
:100680005308C639031908005418DD12D4185D1236
:100690005419DD10D4195D10D31F562B3F1F532B57
:1006A000531F562B7C2B531B562B7C2B5319642B1F
:1006B000D3185D2BBF1B712B7C2B54083E050319EF
:1006C0007C2BDC18712B7C2B54083E0503197A2BEC
:1006D0005C1D7C2B5B085405031D08005408DB04DB
:1006E000712B54188516D418051654198514D4196D
:1006F000051408005408DB0454188512D418051298
:1007000054198510D41905100800701E08008B13A9
:10071000831620088400000883128B1795008B1322
:100720008316A00AAB302002A1300318A000831268
:100730008B1708006430F100E8267208F500E01E0F
:10074000F5016530E01E6030F100E8267208F60021
:100750008B138316A130A0007730A100AD30A2002A
:1007600083128B17AD30761CAF30F61C40388B13DC
:100770008316A30083128B17AD30761DAF30F61DA4
:1007800040388B138316A40083128B17AD30761E6E
:10079000AF30F61E40388B138316A50083128B17DB
:1007A000AD30761FAF30F61F40388B138316A6008E
:1007B00083128B17AD30751CAF30F51C40388B138E
:1007C0008316A70083128B17AD30751DAF30F51D52
:1007D00040388B138316A80083128B17AD30751E1B
:1007E000AF30F51E40388B138316A90083128B1788
:1007F0008330F100E8267203C000AD30401CAF30FA
:10080000C01C40388B138316AA0083128B178B13DE
:1008100083162309A2062409A2062509A206260991
:10082000A2062709A2062809A2062909A2062A0962
:10083000A206AD30A20483128B1708004F08FF3CBC
:10084000D100F0304F07D0008523D401541466083E
:10085000D3004023D401D4146708D3004023D4012B
:1008600054156808D3004023D401D4156908D30077
:100870004023F4242B25C5080319472CDC1F08004E
:10088000DC13DF0B08007D30DF00C50308006608BD
:10089000C639031D4F2C3E1CDD123E18DD166708BD
:1008A000C639031D572CBE1C5D12BE185D166808A4
:1008B000C639031D5F2C3E1DDD103E19DD1469088D
:1008C000C639031D672CBE1D5D10BE195D14DE0BFD
:1008D00008000A30DE00521C8512D21C0512521D7F
:1008E0008510D21D05108524661898246718AC243D
:1008F0006818BE246918D024661C5214671CD214D0
:10090000681C5215691CD21508004B08CA00E22465
:10091000CB004C08CA00E224CC004D08CA004B1C96
:10092000E224CD004E08CA00CB1CE224CE00080011
:10093000C1080319521403190800C60B0800CB1B89
:10094000C1034B08C600CB1852144B195214CB1ECE
:100950005214CB1D52100800C2080319D2140319F7
:100960000800C70B0800CC1BC2034C08C700CC1AF8
:10097000D2144C1DD2144C1FD2100800C308031906
:10098000521503190800C80B0800CD1BC3034D08FE
:10099000C8004D1A52154D1F5215CD1D5211080099
:1009A000C4080319D21503190800C90B0800CE1B8F
:1009B000C4034E08C9004E1AD215CE1FD215CE1D43
:1009C000D2110800C001CA080319CA034A1840140A
:1009D000CA1A40144008C0014A1C4014CA1E4014E0
:1009E000C005C00C4A0C0800D60B0800AF1F102D24
:1009F00003102F1A0314AF0D1F30AF05AF135808A3
:100A00002F02031C092D0319102D2F08D800D50023
:100A1000102D2F08D80065080319D5076308D700E3
:100A20005808640755020318242DDC10E6188512B7
:100A3000E7180512E8188510E91805105808013E56
:100A400055020318252D0800DC14D70B0800630895
:100A5000D700D5030800DA0B0800D90B08008B1368
:100A600083167A309B001C141A088312D9008B1746
:100A70005C1D3C2D5C110800DB015C150800701842
:100A8000582D2A080319462DF301080029080319D7
:100A90004B2DF30108002B080319502DF30108001A
:100AA0002D11F30A06307302031C080070140800AD
:100AB000850187012D112B082A0629020319672DAC
:100AC0002B082A0629062C020319672D08007C3002
:100AD0002B06FC390319E82D701178302B06FC39F0
:100AE0000319862D74302B06FC390319CF2D2B08E2
:100AF000031D812D2A08031D812D2908031D812D29
:100B000008007010F3017012992608007608290277
:100B1000031908002908F600E0307606E039031DC5
:100B200008000130F6180430F50003107618F50DB2
:100B30007619F50E0026F201F019AB2D8B13710812
:100B400083169B001C141A088312F2008B17403086
:100B5000F1080319F200761AB92DF01E0800720888
:100B600075050319B62DF61952260800F61D5226F2
:100B70000800701F080007302A0203190800F61D3C
:100B8000C42D7508F204C62D7509F2058B13710882
:100B9000BC007208BB0057228B1752260800F01EBB
:100BA00008000026F201F019E22D8B13710883165C
:100BB0009B001C141A088312F2008B174030F108B6
:100BC0000319F20072082902031D080052260800CA
:100BD000701908000026701F0800F0190800F108BD
:100BE0000319F22E07302A02031908008B1371082B
:100BF000BC002908BB0057228B177015522608002D
:100C0000F0157013F01A70172B180800AB180800B5
:100C1000F011AA0AF10108302A0203190800603015
:100C2000F10001302A0203190800F10A07302A02F4
:100C300003190800F10A0F302A020319701703196B
:100C40000800F10A10302A0203190800F10A1130D5
:100C50002A0203190800F10A12302A0203190800B7
:100C6000F10AF10AF10A1D302A0203190800303096
:100C7000F4006D30F10074082A0203190800F40A28
:100C80004130740269300319F4006B307402703023
:100C90000319F400A03074020319F01503190800B9
:100CA000F10A3B2EFF308500870031309000003084
:100CB00083168C0083128E018E17FC308F000C106F
:100CC00064000C1C602E0C1085018701013090001F
:100CD000013083168C00831208006830F100E8268A
:100CE0007208E0007A30F100E8267208D9007B3003
:100CF000F100E8267208E3007C30F100E826720873
:100D0000E4007D30F100E8267208E5006D30F10066
:100D1000E8267208E10066308400A630F100E8267B
:100D200072088000F10A840A70300402031C8F2EBE
:100D30000800701A080070166D269A236430F100BE
:100D4000E8267208F500E01EF5016530E01E60300F
:100D5000F100E8267208F6000130F4007408103E35
:100D6000F100E8267608F2020319BC2E8B13BB00B3
:100D70007108BC0057228B177408203EF100E8264A
:100D80007508F2020319CA2E8B13BB007108BC0050
:100D900057228B179B307407F100E82672080F3931
:100DA000F8008027F7007408003EF100E826770875
:100DB000F2020319E12E8B13BB007108BC0057220D
:100DC0008B17F40A0B30740203190800AE2E0800CA
:100DD0008B13710883169B001C141A088312F200EF
:100DE0008B170800F4016030F1008B137108831633
:100DF0009B001C141A088312F2008B177408F80069
:100E0000A027F20203190A2F8B13BB007108BC0044
:100E100057228B17F40A503074020319522EF10A2C
:020E2000F52EAD
:100F000007308A0078088207903481348234843430
:100F10008834B134B234B434B834A134A234A434F3
:080F2000A834813481348134CE
:100F400007308A007808820703343F3401340134C3
:100F5000C034013400340034003400340034003430
:100F60000034003400340034003402340F340434CC
:100F7000FF34FF34FF34FF34FF34FF3405340434CE
:100F800004341034FF34FF34FF34FF34FF340134B1
:100F9000FF34FF34FF34FF34FF34FF34FF34FF34B9
:100FA000FF34FF34FF34FF34FF34FF34FF34FF34A9
:100FB000FF34FF34FF34FF34FF34FF34FF34FF3499
:100FC000013402340334043405340634073408345D
:100FD00009340A34013401348034C034013401341A
:0A0FE0000134013401340134FF3400
:084000000C00000006000300A3
:02400E00CC33B1
:1042000001008100820084008800B100B200B40087
:10421000B800A100A200A400A800FF00FF00FF005A
:104220000300030003000300030003000300030076
:1042300003000300030003000300FF00FF00FF0072
:10424000FF0000000000000000000000000000006F
:1042500000000000000000000000FF00FF00FF0061
:10426000FF00FF00FF00FF00FF00FF00FF00FF0056
:10427000FF00FF00FF00FF00FF00FF00FF00FF0046
:10428000FF00FF00FF00FF00FF00FF00FF00FF0036
:10429000FF00FF00FF00FF00FF00FF00FF00FF0026
:1042A000FF00FF00FF00FF00FF00FF00FF00FF0016
:1042B000FF00FF00FF00FF00FF00FF00FF00FF0006
:1042C00003003F0001000100C000010000000000E9
:1042D00000000000000000000000000000000000DE
:1042E000000002000F000400FF00FF00FF00FF00BD
:1042F000FF00FF000500040004001000FF00FF00A5
:10430000FF00FF00FF000100FF00FF00FF00FF00B3
:10431000FF00FF00FF00FF00FF00FF00FF00FF00A5
:10432000FF00FF00FF00FF00FF00FF00FF00FF0095
:10433000FF00FF00FF00FF00010002000300040077
:10434000050006000700080009000A00010001003E
:104350008000C00001000100010001000100010017
:10436000FF00FF00FF00FF00FF00FF00FF00FF0055
:10437000FF00FF00FF00FF00FF00FF00FF00FF0045
:10438000FF00FF00FF00FF00FF00FF00FF00FF0035
:10439000FF00FF00FF00FF00FF00FF00FF00FF0025
:1043A000FF00FF00FF00FF00FF00FF00FF00FF0015
:1043B000FF00FF00FF00FF00FF00FF00FF00FF0005
:1043C000FF00FF00FF00FF00FF00FF00FF00FF00F5
:1043D000FF00FF00FF00FF00FF00FF00FF00FF00E5
:1043E000AA00FF00FF00FF00FF00FF00FF00FF002A
:1043F000FF00FF00FF00FF00FF00FF00FF00FF00C5
:00000001FF
